:1000000012C02CC02BC02AC029C028C027C026C0BF
:1000100025C062C023C022C021C020C01FC01EC096
:100020001DC01CC01BC011241FBECFE5D4E0DEBF25
:10003000CDBF11E0A0E6B0E0E6E1FBE002C0059034
:100040000D92AA30B107D9F711E0AAE0B1E001C0E2
:100050001D92A238B107E1F77BD05CC5D1CF9C01DE
:10006000832F992780BD29B988E18AB986E880BDA8
:1000700080B5877F80BD08955D9BFECF8CB980E001
:1000800090E00895CF93DF93EC018881882329F0D5
:100090008991F2DF88818823D9F7DF91CF91089584
:1000A0005F9BFECF8CB1992708950F931F93CF9339
:1000B000DF93EC01062F10E006C0101738F48D30E6
:1000C00009F089931F5FECDF8A30B9F71882DF915E
:1000D000CF911F910F9108951F920F920FB60F921B
:1000E00011242F933F934F935F936F937F938F933D
:1000F0009F93AF93BF93EF93FF9380910C018F5F1A
:10010000803958F080B38470682F80E0A0D180B32C
:100110008870682F81E09BD180E080930C01FF9173
:10012000EF91BF91AF919F918F917F916F915F916F
:100130004F913F912F910F900FBE0F901F901895E8
:10014000929A939A81E083BF89B7816089BF0895AD
:10015000CFE5D4E0DEBFCDBF81E090E080DF8FEF60
:1001600087BB11BA8A988B98EBDFE6D080E690E0E7
:1001700047D162E080E025D181E790E041D120E2E3
:100180003EE48CE590E00197F1F721503040C9F74B
:10019000CCD082E890E034D162E080E012D188E8EF
:1001A00090E02ED120E23EE48CE590E00197F1F75B
:1001B00021503040C9F7B9D087E990E021D162E001
:1001C00080E0FFD082EA90E01BD120E23EE48CE5A3
:1001D00090E00197F1F721503040C9F7A6D083EBAA
:1001E00090E00ED162E080E0ECD083EC90E008D1AA
:1001F00020E23EE48CE590E00197F1F72150304099
:10020000C9F793D081ED90E0FBD062E080E0D9D0D7
:1002100082EE90E0F5D061E18EE691E046DF63EF9B
:1002200070E08EE691E067D1892BA9F37ED081E062
:1002300080938101109284017894C09108012C2F41
:10024000332727FD309521303105B9F022303105B3
:100250001CF4232B29F029C02031310529F025C0B9
:1002600080910B018F5F03C080910B018E5F8093A3
:100270000B0199279F938F9305C081E080930B0119
:100280003F932F938DEF90E09F938F930DE011E0BC
:100290001F930F934AD1C801F5DE8DB79EB706961E
:1002A0000FB6F8949EBF0FBE8DBFCF3F19F08FEFF2
:1002B0008093080161E18EE691E0F7DE6DE571E083
:1002C0008EE691E008D1892B09F4B7CF2ED072D0F9
:1002D00080E690E095D062E080E073D08EE691E019
:1002E0008FD06EE671E08DE591E0FED0A6CFAD9A9D
:1002F00081E08A95F1F7AD98089595B3907F95BB0D
:10030000982F92959F7085B3892B85BBF0DF089558
:100310001F93182FAC98F1DF812F8295807FEDDF3E
:1003200083E38A95F1F71F91089581E0F1DF83E37C
:1003300097E00197F1F70895EF92FF920F931F93C3
:1003400084B38F6384BB85B3807C85BB80E096E3F8
:100350000197F1F780E3D1DFE12C82E1F82EC701AC
:100360000197F1F7C4DF09E913E0C8010197F1F73C
:10037000BEDFC8010197F1F780E2BFDFC701019737
:10038000F1F788E2C5DF8CE0C3DF86E0C1DFCDDFB7
:100390001F910F91FF90EF9008951F93182FAC9A23
:1003A000ACDF812F8295807FA8DF88E38A95F1F703
:1003B0001F91089582E0ACDF83E397E00197F1F7A6
:1003C0000895282F862F99278230910579F0833060
:1003D00091051CF4019739F008958330910549F097
:1003E000049751F00895822F805808C0822F8054BE
:1003F00005C0822F805702C0822F805389DF089565
:10040000CF93DF93EC018881882329F08991C5DFA0
:1004100088818823D9F7DF91CF9108950F931F9397
:10042000CF93DF938B01992723E0880F991F2A959B
:10043000E1F780646DDFE80107E08991AEDF0150EC
:1004400007FFFBCFDF91CF911F910F910895482FA8
:1004500083E0489FF0011124E158FE4F918180E034
:10046000662309F481E0682F592F5823892F80953E
:100470008623262F2095292361836FEF3281908177
:10048000882329F0313009F0642F90E00EC0552305
:1004900021F09E3F50F49F5F08C0222331F031309D
:1004A00021F49F3F21F0642F02C0313031F49035A8
:1004B00051F4642F605F9FEF06C0323021F49C330B
:1004C00011F4642F9DE2809108018F3F11F4609335
:1004D000080190830895FB01DC018D910190801942
:1004E0000110D9F3990B0895FB01DC0101900D92E5
:1004F0000020E1F70895FB0151915523A9F0BF01B8
:10050000DC014D9145174111E1F759F4CD010190FE
:10051000002049F04D9140154111C9F3FB014111F3
:10052000EFCF81E090E001970895AEE0B0E0EAE916
:10053000F2E0C7C20D891E892F89388D86E08C8331
:100540001A8309838FEF9FE79E838D83AE01475EF9
:100550005F4FB901CE01019609D02F813885020F76
:10056000131FF8011082E4E02E96C7C2ABE0B0E0A2
:10057000EBEBF2E09BC23C014B015A01FC011782FC
:100580001682838181FD03C08FEF9FEFE8C1F301E5
:100590002381F40123FD059123FF01914F010023E5
:1005A00009F4DAC1053239F423FD059123FF0191E5
:1005B0004F01053229F4B301802F9927E9D1E7CF04
:1005C000CC24DC2C5C2C3AE0FFE1FD1518F1802FE7
:1005D00099278B32910591F08C32910534F4803259
:1005E000910579F0839799F015C08D32910561F0EE
:1005F000C09781F461E0E62EDE2831C052E0F52E8E
:10060000DF2804E0D02A2BC018E0D12A28C040E11E
:10061000D42A25C0D7FC2CC0802F80538A3088F480
:10062000082FD6FE06C0539EC0011124502E580E2E
:1006300016C0C39EC0011124C02EC80E50E2D52A98
:100640000EC00E3229F4D6FC87C180E4D82A07C038
:100650000C3619F490E8D92A02C0083649F4F4019E
:1006600023FD059123FF01914F01002309F0ACCF39
:10067000802F8554833018F08052833038F444E062
:10068000E42EF12CAE0CBF1C8FE316C0802F9927EF
:100690008336910559F08436910524F4833591050C
:1006A00039F158C08337910579F054C0F50102E063
:1006B00010E0A00EB11E808189837E010894E11CA8
:1006C000F11C01E010E011C0F50122E030E0A20EC3
:1006D000B31EE080F180D6FE03C0652D772702C0EF
:1006E0006FEF7FEFC70149D18C013FE7D32213C0E1
:1006F000F50142E050E0A40EB51EE080F180D6FE88
:1007000003C0652D772702C06FEF7FEFC7012AD1A5
:100710008C0150E8D52AD3FC0BC08C2D99270817E3
:10072000190730F4B30180E290E032D1CA94F5CFDA
:100730000115110509F407C1F701D7FC8591D7FE12
:1007400081917F01B301992723D1C110CA9401502F
:100750001040EECF043611F00936A1F5D7FE0BC0DC
:10076000F50134E0E32EF12CAE0CBF1C60817181E9
:10077000828193810EC0F50102E010E0A00EB11E4F
:10078000808191819C01442737FD4095542FCA01F7
:10079000B9013FE6D32297FF09C0909580957095E7
:1007A00061957F4F8F4F9F4F40E8D42A2AE030E079
:1007B000AE014F5F5F4F19D19E012F5F3F4F082F52
:1007C000021B52C0053729F45FEED5222AE030E043
:1007D00027C0E9EFDE228F36910571F08037910551
:1007E00024F488359105A9F0B7C08037910539F018
:1007F0008837910531F0B0C028E030E011C0F0E159
:10080000DF2AD4FE03C024E0E22EDE2820E130E01F
:1008100007C0D4FE03C096E0F92EDF2820E132E0C5
:10082000D7FE0AC0F50104E010E0A00EB11E608101
:100830007181828193810CC0F50142E050E0A40EE9
:10084000B51E808191817C0100271127C801B70165
:10085000AE014F5F5F4FC9D09E012F5F3F4F082F02
:10086000021B8FE7F82EDF20102FD6FE0DC02EEFD3
:10087000D222051548F4152D8D2D992784FF04C02B
:1008800082FD02C03FEED3222D2D332724FF0DC061
:10089000FE01E00FF11D8081803319F449EED4226E
:1008A00008C01F5F22FF05C003C08D2D867809F0A8
:1008B0001F5FED2CFF24E3FC11C0E0FE07C0502EAB
:1008C0001C1520F45C2C511A500E1C2D1C1530F4F4
:1008D000B30180E290E05CD01F5FF8CF1C1518F4E4
:1008E0008C2D811B01C080E0C82EE4FE0FC0B30137
:1008F00080E390E04DD0E2FE14C0E1FE03C088E545
:1009000090E002C088E790E0B3010AC08D2D8678A0
:1009100041F080E2E1FC8BE2D7FC8DE2B301992744
:1009200037D0051530F4B30180E390E031D05A940C
:10093000F8CF0150FE01E00FF11D8181B30199272D
:1009400027D00023B1F7CC2009F421CEB30180E2F7
:1009500090E01ED0CA94F7CFF30186819781EFE033
:100960002B96C0C0FC010590615070400110D8F773
:10097000809590958E0F9F1F0895FC0161507040E7
:1009800001900110D8F7809590958E0F9F1F0895C4
:100990000F931F93CF93DF938C01EB018B819927EA
:1009A00081FF1CC082FF0DC02E813F818C819D8103
:1009B0002817390764F4E881F9810193F983E88302
:1009C00006C0E885F985802F0995892B39F48E8139
:1009D0009F8101969F838E83C80102C08FEF9FEF96
:1009E000DF91CF911F910F910895FA01AA27283026
:1009F00051F1203181F1E8946F936E7F6E5F7F4FEC
:100A00008F4F9F4FAF4FB1E03ED0B4E03CD0670F67
:100A1000781F891F9A1FA11D680F791F8A1F911DBA
:100A2000A11D6A0F711D811D911DA11D20D009F40A
:100A300068943F912AE0269F11243019305D31934C
:100A4000DEF6CF010895462F4770405D4193B3E035
:100A50000FD0C9F7F6CF462F4F70405D4A3318F0DC
:100A6000495D31FD4052419302D0A9F7EACFB4E08D
:100A7000A6959795879577956795BA95C9F7009745
:100A80006105710508959B01AC010A2E06945795E6
:100A9000479537952795BA95C9F7620F731F841F3D
:100AA000951FA01D08952F923F924F925F926F92D3
:100AB0007F928F929F92AF92BF92CF92DF92EF92EE
:100AC000FF920F931F93CF93DF93CDB7DEB7CA1B6F
:100AD000DB0B0FB6F894DEBF0FBECDBF09942A889A
:100AE000398848885F846E847D848C849B84AA8442
:100AF000B984C884DF80EE80FD800C811B81AA81CF
:100B0000B981CE0FD11D0FB6F894DEBF0FBECDBF99
:060B1000ED010895FFCF86
:100B16002A2A205769666920526164696F202A2A49
:100B26000077756C66662D776F657374656E2E64D7
:100B36006500496465653A0053656261737469616D
:100B46006E205061756C00556D7365747A756E67AD
:100B56003A004672696564656D616E6E20572E2D8A
:100B6600572E005370656369616C207468616E6B03
:100B7600733A004B6172796E61204B72796E6B6FBE
:100B8600003E3E3E2056657262696E6465203E3EBA
:100B96003E003E2042697474652077617274656E0A
:100BA600203E004156522053746172740074756E73
:0A0BB60065723A2025640A00FF0072
:00000001FF
